S00C0000446F6F722E7372656384
S11300000C9434000C943E000C943E000C943E007E
S11300100C943E000C943E000C943E000C943E0064
S11300200C943E000C943E000C943E000C943E0054
S11300300C943E000C943E000C943E000C943E0044
S11300400C943E000C943E000C943E000C943E0034
S11300500C943E000C943E000C943E000C943E0024
S11300600C943E000C943E0011241FBECFEFD4E04C
S1130070DEBFCDBF0E9440000C9456000C940000DB
S113008084B1836084B9289A21E092E085B1822703
S113009085B985B1892785B93FE744E88EE13150B8
S11300A040408040E1F700C00000F0CFF894FFCF5B
S9030000FC
